:020000040800F2
:10000000C81B0020A9010008F50E0008E106000841
:1000100000000000000000000000000000000000E0
:100020000000000000000000000000003512000881
:100030000000000000000000F70E00083513000863
:10004000BB010008BB010008BB010008BB010008A0
:10005000BB010008BB010008BB010008BB01000890
:1000600000000000BB010008BB010008BB01000844
:10007000BB010008BB010008BB0100080000000034
:10008000BB010008BB010008000000003914000893
:100090006D140008D114000805150008BB01000804
:1000A000BB010008BB010008BB0100086515000882
:1000B000F51500080000000000000000000000002E
:1000C000BB01000800000000BB01000800F002F8BE
:1000D00000F03EF80CA030C8083824182D18671E10
:1000E000A246AB4654465D46AC4201D100F030F822
:1000F0007E460F3EB6460FCC0126334200D0FB1A97
:100100003343A246AB4618477838000098380000C1
:10011000103A02D378C878C1FAD8520701D330C850
:1001200030C101D504680C60704700000023002432
:1001300000250026103A01D378C1FBD8520700D31E
:1001400030C100D50B6070471FB51FBD10B510BD85
:1001500000F0AAF81146FFF7F7FF02F0B7F900F038
:10016000C2F803B4FFF7F2FF03BC00F0C9F80000C7
:1001700070B505460C46164602E00FCC0FC5103E82
:10018000102EFAD2082E02D303CC03C5083E042E4B
:1001900007D301CC01C5361F03E021782970641C08
:1001A0006D1C761EF9D270BD07488047074800478E
:1001B000FEE7FEE7FEE7FEE7FEE7FEE70448054947
:1001C000054A064B7047000049130008CD0000089F
:1001D000C8130020C81B0020C8170020C817002023
:1001E000F8B5042A2CD3830712D00B78491C03706E
:1001F000401C521E83070BD00B78491C0370401C17
:10020000521E830704D00B78491C0370401C521EF9
:100210008B079B0F05D0C91ADF002023DE1B08C9FE
:100220000AE0FFF7A5FFF8BD1D4608C9FD401C46C2
:10023000B4402C4310C0121F042AF5D2F308C91A87
:10024000521EF0D40B78491C0370401C521EEAD495
:100250000B78491C0370401C012AE4D40978017012
:10026000F8BD01E004C0091F0429FBD28B0701D5AA
:100270000280801CC90700D00270704700290BD093
:10028000C30702D00270401C491E022904D3830711
:1002900002D50280801C891EE3E70022EEE70022DF
:1002A000DFE7704770477047754600F025F8AE46A7
:1002B000050069465346C008C000854618B020B501
:1002C000FFF77CFF60BCB64600260027C0C5C0C54E
:1002D000C0C5C0C5C0C5C0C5C0C5C0C5403D490832
:1002E00049008D46704710B50446C046C0462046BA
:1002F000FFF737FF10BD0000004870479000002056
:1003000001491820ABBEFEE726000200704700003E
:10031000B0B588B0994802F0DBFC40F2005002F022
:10032000D7FC0024204601F0C1FA01AD40F20010D4
:100330002883AC760E4901910E49891C039140F245
:1003400000410491029042F20000069008200590BE
:10035000204601F0A3FA2046294601F0D1FA2046B2
:1003600001F006FB204601F091FA08B0B0BDC0468E
:100370004C2401404801002070B514460D46064645
:10038000200407D0B0B200F007F82870641E6D1C7E
:10039000761CF5E770BD000070B5044600F056F914
:1003A000A020214DA847214EB047200AA847B047BA
:1003B000E0B2A847B04700F049F9A120A847B047EC
:1003C000002000F08FF9044600F060F9204670BD6F
:1003D00070B514460D460646200407D02978B0B201
:1003E00000F006F8641E6D1C761CF5E770BD000079
:1003F000F8B50C46054600F029F9A0200A4EB04792
:100400000A4FB847280AB047B847E8B2B047B847DC
:100410002046B047B84700F039F90A20F8BC02BCC2
:100420008E4600F0BBB8C04649070008AD0700087B
:10043000F0B50B4D00210B4A0B4B0C4684420DD0FE
:10044000165D75400E46072E06D86F08ED0700D0E2
:100450005F403D46761CF6E7641CEFE7A8B2F0BDAE
:10046000FFFF0000AD0A002001A000009B48002112
:100470008170704799480021C1707047F0B587B00E
:1004800040F2005011303C4CA04740F20050123076
:10049000A0473A48A04740F20050A04706200590E8
:1004A00002F024FB09200690C006032404940025D2
:1004B000F32321462A4601F0C9FF314821462A4646
:1004C000234601F0C3FF01F01DF9FFF721FF0126CC
:1004D00040F20010314601F0ABF9022001903146A4
:1004E00001F0A6F9072003904104304601F02AF9F3
:1004F000284601F0FBF8284601F07EF90821029118
:10050000304601F0D3F805241E4F284629462246DE
:10051000B847304631462246B84704250198294657
:100520002246B847049821462246B8472846059DEA
:1005300029462246B8472046039F39462246114B9A
:1005400098472846029922460E4DA84738460699F4
:100550002246A84701F0ECF801F0EAF801F096F81D
:1005600001F0DEF8304601F051F9304607B0F0BC3A
:1005700002BC8E4601F04AB9D12C000809060000E1
:10058000000400486D17000828B10349414343F2B5
:100590000000B1FBF0F07047E880000081B00090EF
:1005A00003480099016001680029FCD101B070473F
:1005B000F00A002081B00090009801B07047F8B5B3
:1005C00005460920C406204640F6000101F033FF2D
:1005D000204641F2000101F02EFF00270126082FDE
:1005E00020D02846F840C00705D0204648F2000138
:1005F00001F023FF04E0204648F2000101F01BFF58
:100600003046FFF7D7FF204640F6000101F015FF06
:100610003046FFF7CFFF204640F6000101F00BFF08
:100620007F1CDCE701252846FFF7C4FF204641F286
:10063000000101F002FF2846FFF7BCFF204641F20F
:100640000001F8BC04BC964601F0F5BEF8B500F018
:100650003DFE834C01262046314601F0EEFE022588
:100660002046294601F0E9FE04273846FFF7A2FF9D
:100670002046314601F0DFFE3846FFF79BFF20465B
:100680002946F8BC04BC964601F0D5BEF8B500F08A
:100690001DFE734C02252046294601F0CCFE0126A2
:1006A0002046314601F0C7FE04273846FFF782FF97
:1006B0002046294601F0C1FE2046314601F0BDFE2C
:1006C0003846F8BC02BC8E46FFF774BF03488078FA
:1006D0007047C0460148C0787047C046F00000200F
:1006E000FEE70000FEB5009000F0EAFD00210226C2
:1006F000012001900C46019D07291CD8584F38460F
:100700000291314601F097FE3046FFF753FF38461D
:10071000314601F092FE3846294601F092FE274606
:1007200004462846FFF746FF0299601E8441780080
:100730000419491CE0E7009810B100F083FD01E0C6
:1007400000F0A0FDE0B2FEBDFEB5044600F0BEFD27
:1007500043480226314601F06EFE00270120019039
:10076000072F1FD860B2002802943D4D284603D4BD
:10077000019901F060FE02E0019901F05EFE304651
:10078000094CA0472846314601F057FE3046A047A5
:100790002846314601F04FFE3046A0477F1C029CA0
:1007A0006400DDE7FEBDC046B505000870B500F089
:1007B00087FD2B4C0221204601F03FFE01252846F3
:1007C000FFF7F8FE00262046294601F03AFE30B138
:1007D000701CFA2E0646F6D3FFF758FF04E00221FC
:1007E000204601F028FE0025284670BDC046C046C0
:1007F000F8B5394802F06CFA384801250024934EC8
:100800002946224648F20003B0470326904F33485A
:100810002146324648F20003B847304848F200010A
:1008200001F009FE2C48C01C02F052FA0C4829467F
:1008300022462B46854FB8470948214632462B466B
:10084000834FB84702270648294622463B467F4D3C
:10085000A8470348214632463B467D4CA047F8BD99
:1008600000140048F8B5774802F032FA764C0025BB
:1008700001261023754F204629463246B8472023CB
:10088000204629463246B84740232046294632466C
:10089000B8478023204629463246B847F8BDC046AF
:1008A000B0B50D4802F014FA0C4C01210025204689
:1008B0002A4642F2000301F0C9FD032220462946E0
:1008C00042F2000301F0E1FD204642F20001B0BC1B
:1008D00004BC964601F0AFBD1305000000080048B7
:1008E00070470000F0B585B0564802F0F1F9564C5B
:1008F000012103910227554D20463A46049740F2C4
:100900000013A84700210291032520462A4601959D
:1009100040F200134E4EB047204640F200114D4ABF
:1009200090472046039E31463A4640F20023F14F5D
:10093000B8472046029F39462A4640F20023444DDC
:10094000A847204640F20021424A904720463146BF
:10095000049E324640F20043E64DA8472046394601
:10096000019A40F200433A4DA847204640F2004128
:10097000384A904720460399324640F60003DD4D41
:10098000A84720463946019D2A4640F60003304ECE
:10099000B047204640F600012E4A90472046039E6D
:1009A0003146049A41F20003D24FB84720460299DB
:1009B0002A4641F20003FB4FB847204641F20001AE
:1009C000F94A904720463146049E324642F20003DF
:1009D000F34FB847204602992A4642F20003F14FEE
:1009E000B847204642F20001EF4A90472046039F55
:1009F0003946324644F20003E94EB0472046029E93
:100A000031462A4644F20003E64DA847204644F208
:100A10000001E54A904720463946049A48F200030F
:100A2000DF4DA84720463146019A48F20003DD4DCC
:100A3000A847204648F20001DB4A05B0F0BC08BCDC
:100A40009E46104712050000000400484D2400088F
:100A50008B240008372400080C48006840F2E83175
:100A6000B0FBF1F0401E010E00D0FEE70849094A34
:100A70005060094803680B40032189075918016039
:100A800000209060072010607047C04604000020DE
:100A9000FFFFFF0010E000E020ED00E0F0B587B0C0
:100AA00037480021017081600E460191354940F2BE
:100AB00010608847344D35492846884703AC34498F
:100AC00020468847472002902080324805900496AF
:100AD000314A2846214690470127304A2846394660
:100AE00000979047142002212D4A90472D4928460F
:100AF000884740F21060401C224988472A4E304601
:100B00002249884703AD2846214988470298288012
:100B100020480590019C0494304629461E4A90477F
:100B2000304639461D4A90471520032529461C4A60
:100B3000904730461B49884740F21060801C11499D
:100B400088471A4E30461149884703AF3846104946
:100B5000884717483880174805900494304639462E
:100B60000D4A9047304600990C4A90471620294676
:100B70000B4A904730460B49884707B0F0BDC04646
:100B8000F0000020D12C0008004001406D2D00082D
:100B9000C12E0008E7030000E12D00089D2E00088B
:100BA000552A0008D72D00080044014000480140A4
:100BB0001F1C00000F270000FEB502901C2002271A
:100BC0003946009701F046FF744802F081F8092089
:100BD000C50601240426019628462146324601F026
:100BE000FFFB284639462246334601F02FFC0027FA
:100BF000284639462246334601F047FC0826284657
:100C00002146324601F0ECFB284600992246334645
:100C100001F01CFC284639462246334601F035FCDB
:100C2000144802F055F8144C204602F09FF9204673
:100C3000029902F069F92046394602F011FA20467D
:100C4000394602F022FA2046394602F0F4F92046ED
:100C5000019902F0FDF92046314602F00EFA2046D5
:100C600002F09EF90521204603B0F0BC04BC964674
:100C700002F0B4B91107000000440040F8B51B4C65
:100C8000204602F025F8204602F022F8184F0124F1
:100C90004025434E3846214622462B46B047002683
:100CA00003220092384631462B4601F0EEFB3846CF
:100CB000294601F0C0FB02228025384621462B46FA
:100CC000374FB8470A4F38463146009A2B4601F055
:100CD000DCFB3846294601F0B0FB85483146224608
:100CE00044F200032E4CA047F8BDC0461605000094
:100CF000001400484D240008FEB5284801F0E8FF24
:100D00000920C40601260025254F204631460296BB
:100D10002A4640F60003B84703220192204629469E
:100D200040F600031F4FB847204640F600011E4A18
:100D30009047204631462A4641F20003184EB047FC
:100D400020462946019F3A4641F20003154EB0471E
:100D5000204641F20001144A9047204602992A4653
:100D600048F200030E4EB047204629463A4648F264
:100D700000030C4DA847204648F200010A4A90475C
:100D8000204640F60001084A9047204641F2000103
:100D9000054A03B0F0BC08BC9E4610471105000090
:100DA0004D2400088B240008372400080248002145
:100DB0004170FFF763BBC04648010020F0B58DB01D
:100DC00005A82021FFF76BFA0024022520462946BA
:100DD00000F08CFD0028F9D000200221049000F0E2
:100DE0007BFD4C203B493C4B5C2805D00A184C3A13
:100DF00012881A52801CF7E70120374A5070C04C05
:100E00003649C91C039111460A220292944A13469C
:100E1000C833019328320092002858D0087938B19D
:100E20000020087101204821082200F047F92A49D2
:100E30002078002849D0049921700398082913D0FC
:100E40008A0005AB9A18002318241F46042B07D0EC
:100E5000F8252540C65CAE40F719F8345B1CF5E771
:100E60001760001D491CE9E70698029BB0FBF3F0F0
:100E70000799B1FBF3F1184A9061D1610598B0FB75
:100E8000F3F077498860164989780022009B019C1D
:100E9000072A15D01860012797402568A84202D874
:100EA000256CA84207D2FDB229430D4DA97010331D
:100EB000241D521CECE70F42F9D0B943C9B2F4E744
:100EC0000020054948708E4CA6E74878A4E70DB08D
:100ED000F0BDC0464A010020300200207F01002002
:100EE00000000020024842F2000101F0A8BAC0460A
:100EF0000008004870477047F0B587B00024574D90
:100F00002046294640F20012FFF736FA287808B149
:100F1000082802D3514907200870697840F2C812A6
:100F20004F4B9950E97840F2D01299504D490870D2
:100F30000695072C00D182E0611D685C08B1642829
:100F400001D30020685422461532A95C09B16429F6
:100F500001D30021A9540194A200414BD31840F2BF
:100F60001822995040F2D811585040F288101818A1
:100F7000049040F248101818059040F20810181814
:100F80000290C83303930320C44300201822034671
:100F900006460146A4B1069D2F19BD257D5D9540ED
:100FA00028188D257D5D9540EB185D257D5D95406C
:100FB000AE192D257D5D95406918083A641CE9E756
:100FC000029A1660039A1160059A1360049A1060E1
:100FD000254A914202D3264CA14202D92449039CBE
:100FE00021609642019C1D4D02D3214FBE4202D981
:100FF000029E32601646B14203D2029A11600399F2
:101000000E6040F2F4118B4202D3184A934202D987
:10101000164B059A1360884202D3144A904203D9B2
:101020000498016040F2F410834203D204990B60EB
:10103000059908600698001D0690641C79E7252034
:101040000649085C40F25822054B98502720085C5E
:1010500040F25C21585007B0F0BDC046AC050020FE
:101060008C02002001000020E02E0000905F0100B3
:10107000D0DD060070B56E4C10210E4E2046B047F4
:101080000D4D287020212046B04768704021204631
:10109000B047A87080212046B047C000A9788900D9
:1010A0000143687840000843297801430F208843B2
:1010B00070BDC0463712000844010020B0B5104B87
:1010C00000251D700F4B1D700F4C62712571E17072
:1010D00003236370207090000C4A1070090AA170FD
:1010E000401D0B4908700620FFF7A2F9A071000A05
:1010F000E07108212046B0BC04BC964600F002B95D
:101100007E0100207C010020AD0A0020AC0A0020F6
:101110007D010020B0B5464C07283DD8820001A3D0
:101120009A18974600F00EB800F012B800F016B802
:1011300000F01AB800F01EB800F022B800F051B864
:1011400000F024B82046012955D140F200114DE0AD
:101150002046012952D140F2002147E020460129D2
:101160004FD140F2004141E0204601294CD140F6E8
:1011700000013BE02046012949D141F2000135E060
:101180002046012946D142F200012FE020460129E4
:1011900043D148F2000129E0394D204640F20011C8
:1011A000A847204640F20021A847204640F20041CF
:1011B000A847204640F60001A847204641F200011A
:1011C000A847204642F20001A847204644F2000109
:1011D000A847204648F200012A46B0BC08BC9E46FB
:1011E0001047204601291BD144F20001B0BC04BCC9
:1011F000964601F022B940F2001113E040F20021BE
:1012000010E040F200410DE040F600010AE041F23A
:10121000000107E042F2000104E048F2000101E0B1
:1012200044F20001B0BC04BC964601F004B9C046CB
:1012300000040048704780B501F003F9411E884161
:1012400080BD000070B52D4C02250D4E204629466C
:10125000B04700F03BF801212046B0472846FFF791
:10126000A9F92046294601F0E8F82846FFF7A2F937
:1012700020462946324670BC08BC9E461047C046F0
:1012800037240008B0B51D4C02252046294601F040
:10129000D2F800F01BF80121204601F0CEF82846D4
:1012A000FFF788F92046294601F0C7F82846FFF7DE
:1012B00081F920462946B0BC04BC964601F0BBB873
:1012C000F148002101230A4601F0C0B870B5EE4C88
:1012D00000250126204631462A46334601F0B6F85D
:1012E000032220462946334601F0CFF8044848F24D
:1012F000000170BC04BC964601F09DB80014004883
:1013000000080048F8B50C4600900025C84E084F6C
:10131000A5420CD00098415D304601F021FE3046D8
:10132000394601F04AFE0028F9D06D1CF0E7F8BDFF
:10133000060700000348016811B10168491E0160F9
:101340007047C046F00A002030B4334802680121DB
:101350000A43026002689207FCD542682F4B134093
:10136000436042682E4B1340436002682D4B13408C
:101370000360C26A0F239A43C262026B40F20313F6
:101380009A4302630A04036B93430363CA07036B24
:1013900093430363426B8A43426300228260036883
:1013A0000B430360204B5B1E144654410568AD0798
:1013B00001D4002CF7D10268920700D4FEE71B4B42
:1013C0001A680724A2431A601C68022214431C6096
:1013D0004368436043684360436843604368144C18
:1013E0001C4044604368134C1C4344600B06046873
:1013F0001C43046003689B01FCD543680324A3439A
:10140000436043681343436042681207FCD5C80633
:10141000002130BC01F04ABB001002400C00FF0864
:10142000FFFFC277FFFFF2FEFF0400000020024032
:10143000FFFFC2F70000040810B50A4C0121204646
:1014400001F034FD68B10121204601F02BFD00219F
:10145000204601F089FC0448006810BC02BC8E469E
:10146000004710BD0020004020020020F8B5154DB7
:1014700001242846214601F019FD012803D101214C
:10148000284601F00FFD3449283100220E4B0F4D44
:10149000072A10D09E5C5EB10E461C3E3768086875
:1014A000874201D2781C02E0AC540020985430608E
:1014B000091D521CECE7284A916809B1481E90604A
:1014C000F8BDC046004001405002002065020020E7
:1014D000B0B50B4D01242846214601F0E7FC012858
:1014E00003D10121284601F0DDFC1B488188491CFD
:1014F000818089B2642902D3002181808470B0BDCB
:1015000000440140B0B5134D01242846214601F0A6
:10151000CDFC012803D10121284601F0C3FC0E486F
:10152000C4700178042901D8491C02E00B490C70F1
:10153000002101700A490A7822B14278092A04D8A8
:10154000511C00E000214170B0BD00220A704270C1
:10155000B0BDC04600480140F00000203402002029
:1015600031020020B0B51D4C324D2046294601F015
:1015700053FD30B11A48006880472046294601F0E3
:1015800037FD184D2046294601F017FD012806D1E8
:101590002046294601F009FD114800688047124D98
:1015A0002046294601F038FD30B1104800688047D8
:1015B0002046294601F01CFD0D4D2046294601F02C
:1015C0002BFD48B109480068804720462946B0BC39
:1015D00004BC964601F00CBDB0BDC04600380140C9
:1015E0001802002003070000070007071C02002064
:1015F00006000607B0B50E4C0E4D2046294601F0F8
:101600000BFDA0B12046294601F0F2FC204601F076
:10161000A3FC09490A78531C0B708A18D0704878CB
:10162000DAB2824203D30120887000200870B0BD76
:1016300000440040050005077C010020B0B50020F3
:10164000064CA047064D28600120A0476860022094
:10165000A047A8600320A047E860B0BDB12B0008F8
:1016600034010020B0B5084C80252046294600F002
:10167000E4FE2046294600F0DEFE20462946B0BCA6
:1016800004BC964600F0D9BE0014004867480168C3
:1016900008220A43026001680907FCD40168042299
:1016A0000A43026001684907FCD4704702280ED043
:1016B000012818D10F2000050B4A136883431360DB
:1016C000090509180140106808431060704703209D
:1016D0000005054AD3688343D36009050918014012
:1016E000D0680843D06070472C240140411E8841D7
:1016F000C0024E490A6840F600039A431018086079
:101700007047C04610B5054C204601F0F5FA20465A
:1017100010BC02BC8E4601F0E5BAC04609030000C9
:101720004248016840F200120A4302607047C04616
:101730003E480168C90703D1016801220A430260DB
:101740007047C046012803D0022809D1064800E0AE
:101750000448364A13680340136010680843106059
:101760007047C046FFFFF1FFFF8FFFFFB0B5214B71
:1017700005280AD8052444430846A0401F25A54053
:101780009C6AAC4304439C621AE00B280BD80524E6
:1017900044431E3C0846A0401F25A5405C6AAC435C
:1017A00004435C620CE010280AD2052444433C3C0C
:1017B0000846A0401F25A5401C6AAC4304431C6298
:1017C000092909D8032048438240072181405868ED
:1017D000884310435860B0BD122909D803204843FC
:1017E0001E388240072181401868884310431860E2
:1017F000B0BDC0460C24014003210906224A1368EB
:101800008B4313601168014311607047C10707499A
:1018100004D0012292050B6813430B60800704D5A6
:10182000012040050A6802430A607047082401400D
:1018300010B540F2001304461C40134A81B114B1A4
:10184000116819431160410504D540F20041136845
:101850000B431360800716D551680220084311E03E
:1018600024B1116840F2001399431160410504D579
:10187000116840F2004399431160800703D5506816
:1018800002218843506010BD0424014014214143CB
:101890003C480A58012313430B507047142141431D
:1018A00038480A58202313430B50704710B51422B0
:1018B00042430D49521853680124A3435360002347
:1018C00053609360D360136180000F2282400868E8
:1018D0001043086010BDC046800081400248026885
:1018E0000A4302607047C046040002408000814005
:1018F000024800680840411E8841704700000240CD
:10190000B0B5142242431F4813580124A343135077
:1019100013180C689C608C68DC600C8A5C6013583F
:1019200043F60074A3434C681C43CB6823434C69C3
:101930001C4314500B7E5B1E5C425C41A301145897
:101940004025AC43E31813504B7E5B1E5C425C4168
:10195000E30114588025AC43E3181350897E4B1ED5
:101960009941090113581024A34359181150B0BDCF
:101970001421414303480A5844F200039A430A5091
:101980007047C0460800024010B5144608463F495B
:101990000A220A700722214601F02CFD012804D1F9
:1019A000044801F0A1FD012801D0032010BD002052
:1019B00010BDC046204E0000F8B506460F4CA0886A
:1019C000000A16D1A0880527032810D30D460092DF
:1019D000A188264801F07FF848B92449087830707A
:1019E000481C2860A088801E00990880002738467F
:1019F000F8BD03A00C499C22FFF748FEC00100205F
:101A00007573526376427566666572506F73203CDB
:101A1000204D425F5345525F5044555F53495A45EC
:101A20005F4D415800000000E4380008B0B5174D84
:101A30006B780BB1052516E00124EC804B1EAB60E2
:101A40001870E8888018E880E988184601F043F8A3
:101A5000E9884A1CEA80054A5054AC7000252846A3
:101A6000214601F01FFB2846B0BDC046F40A002005
:101A700010B501200024214601F014FB03484470F6
:101A8000204610BC02BC8E4601F0A2BCC001002062
:101A900080B50020014601F005FB80BC01BC8646F4
:101AA00001F034BB10B5064C2078012805D105485B
:101AB000806880470020207010BD062010BDC04601
:101AC0000800002000020020F8B50D460988032414
:101AD00005292CD10279C17809028E18711E89B2AC
:101AE0002E4B994223D88178437800242C800127FB
:101AF00007702F887F1C2F805707B2B2D60807B116
:101B0000761C46702F887F1C2F801B025918491C99
:101B100089B2801C234600F0E1FA20B1F8BC02BC77
:101B20008E4600F0CDBFF0B22988081828802046E4
:101B3000F8BDC046F8B50D460988032405292BD108
:101B40000279C17809028E18711E89B2134B99422D
:101B500022D88178437800242C80022707702F88B0
:101B60007F1C2F805707B2B2D60807B1761C46708B
:101B70002F887F1C2F801B025918491C89B2801C9A
:101B800000F004FB20B1F8BC02BC8E4600F098BF08
:101B9000F0B22988081828802046F8BDCE0700003A
:101BA000F8B50C4609880325052922D10279511E72
:101BB0007C291ED88178437800252580032606706D
:101BC0002688761C26805600467027887F1C278032
:101BD0001B025918491C89B2801C2B4600F0FCFAE4
:101BE00020B1F8BC02BC8E4600F06ABF2088801984
:101BF00020802846F8BDF8B50D460988032405293C
:101C000026D10179C278120251184A1E92B27B2A5B
:101C10001ED88378477800242C80042202702A88FA
:101C2000521C2A808AB2560046702988491C298095
:101C30003902C918491C89B2801C00F0B7FB20B1D9
:101C4000F8BC02BC8E4600F03BBF28888019288073
:101C50002046F8BDF8B5054608880A2841D30C4649
:101C60002879E97809020F18781E80B203267C28AB
:101C700038D8287AE97909020818010432D082B2EA
:101C8000792A2FD8687A510088422BD1A8796979AE
:101C900009020818411CA87800906E7828460A307E
:101CA00089B2012300F098FAB0B9BAB230020099B3
:101CB0004018411CA81C0026268017232B7023885F
:101CC0005B1C238057006F7023885B1C238089B2C4
:101CD000334600F081FA38B1F8BC02BC8E4600F001
:101CE000EFBE00263046F8BD2088C0192080F9E7F5
:101CF000B0B50C4605490D88401C891C2A46FEF7E4
:101D00006FFA681C20800020B0BDC046D0010020C2
:101D10001CB50988032405291AD10179C1B9827833
:101D20004378C178FF2900D091B918028018421C6D
:101D300001A800244470FF394B424B41037091B21B
:101D40000122134600F0CAF910B100F0B9FE0446B2
:101D500020461CBD80B50988052910D181784278BC
:101D600012025118491C89B2C01C0122134600F00E
:101D700033FA30B180BC02BC8E4600F0A1BE032015
:101D800080BD002080BD70B50C460A880321062A5C
:101D900024D30679C27812029519AAB2D30876071D
:101DA00000D05B1C6D1EADB22D097A2D16D8457979
:101DB000DBB29D4212D1817843781B025918491C2D
:101DC00089B2801D012300F089F920B170BC02BCEA
:101DD0008E4600F075BE052020800021084670BDAB
:101DE000B0B50C46014622880320062A20D30B7981
:101DF000CA781202D218551EADB2772D18D84D7977
:101E00005B061B0E9D4213D188784B781B02181875
:101E1000431C881D99B292B2012300F0DDF920B174
:101E2000B0BC02BC8E4600F04BBE052020800020D6
:101E3000B0BD0000F8B50546022091B3CC081E2CB9
:101E40002FD8069C524E3170012D15D04DBB254D1B
:101E50002548264FB760F0603561214870611F4802
:101E6000B0611D48F0611B483062084611461A46B1
:101E7000234600F091F813E0134D1448144FB76057
:101E8000F06035610F4870610D48B0610B48F0613A
:101E900009483062084611461A462346FFF774FD8A
:101EA00000B1F8BD01F08EFA20B13848012101706F
:101EB0000020F8BD0320F8BD79320008B1320008D7
:101EC0006D310008B91900082D1A0008911A000890
:101ED000711A0008D135000819360008413500088C
:101EE000D51F000849200008C9200008AD200008BF
:101EF0007CB52648007808B1062445E001A801F029
:101F000055FA002401283FD101A80078022812D0F8
:101F1000012839D11E4D6B69681C294624312A1DC0
:101F2000984788BB68782978884200D060BB022037
:101F300001F04EFA28E0164D6A6A1178A970002364
:101F40000120144C802B0AD0E65C46B18E4201D0B1
:101F50000833F7E7E0184368291D10469847697869
:101F6000002489B158B10121A980A97880220A43AF
:101F7000696A0A70A9884A1CAA806A6A5054AA88A9
:101F8000696A28782B69984720467CBD08000020A4
:101F9000000200200C00002010B51446084608225C
:101FA000214601F027FA01280ED144F60030844280
:101FB00001D9232003E060000549B1FBF0F080B2B5
:101FC00001F092FA012801D0032010BD002010BDBD
:101FD000A07F1700F8B506460F4C6088000A16D19E
:101FE00060880527042810D30D46009261882E488A
:101FF00000F070FF48B92C4908783070481C286000
:102000006088C01E0099088000273846F8BD03A0EC
:102010000C499C22FFF73AFBF401002075735263D0
:1020200076427566666572506F73203C204D425F44
:102030005345525F5044555F53495A455F4D41588F
:102040000000000065390008B0B51E4D2B78012B4B
:1020500026D10124AC804B1EAB601870A888801874
:10206000A880A988184600F035FFA9884A1CAA80D4
:102070000D4A5054A9884B1CAB80000A5054A868E4
:10208000007801F027FAA888401EA880A868401CA4
:10209000A8606C7000252846214601F003F800E096
:1020A00005252846B0BDC046F40A002080B5054885
:1020B00000210170012000F0F5FF80BC01BC8646C4
:1020C00001F03CB8F401002080B50020014600F08A
:1020D000E9FF80BC01BC864601F018B8FFB5044694
:1020E000491E88B28018042829D8501E0825019559
:1020F00090FBF5F0451C00201BB3012B42D1009052
:102100000123214F28043CD06D1E029503942478AE
:10211000019DE8B2464246411004184600D03046C0
:10212000521E40B9012020408EB2B855491C6D1E88
:10213000E0B24408EDE7039C641C029DE2E7012045
:1021400020E00090012728041BD003946D1E029507
:1021500008240025E6B27042704116043E4600D0C5
:102160000646521E46B988B2074E305CA84003436B
:102170006D1C491C641EEDE7039C2370641C029DCA
:10218000E1E7009804B0F0BDF40B0020F0B5491E63
:102190008BB2DC0801217D2C1BD39B1840F2EC3460
:1021A000A34216D8511E082391FBF3F14C1C0021C9
:1021B00025040ED0641E16461D46721E360404D039
:1021C0006F1E2D0616463D46F7D100250570401CB2
:1021D000EEE70846F0BD0000FEB50F460646481E75
:1021E00084B2012063498C4200D8C2E01546A11890
:1021F000614A914200D9BCE041F27071621A5F49B4
:102200004A60012B0CD00BBB5A48401C844259D168
:10221000022D57D1500060490968594A115261E0B6
:10222000019200904D7062005548121842F6E0632A
:10223000D21A2B4619040BD031780902118070781C
:1022400008181080B61C921C5B1EF3E70020FEBD30
:102250004848401C844247D1019840004849091829
:102260002806C20D4C4C2046FDF7BAFF206808B185
:10227000082801D30720206002AE30700025012716
:10228000284631463A46FEF7A3F8307843490870AD
:102290000821081AFF21C140414C217038463146BF
:1022A0003A46FEF769F82078029901403D48C1732B
:1022B000394B186840F20072801818603A48017073
:1022C0002846FEBD41F2A370381A303080B29528FE
:1022D00039D850002A49081891002F4A51186A002D
:1022E000FDF77EFF00222FE041F2A370381A80B282
:1022F00065280098019A3CD85000214909181F48C8
:102300000078009046011F488419204608302A06AC
:10231000D20DFDF765FF01201A49885101996160CE
:102320000099491CCAB200231F2A1C461A4600D82D
:102330000A4612490A7014498F4217D013498F4236
:1023400016D1144913E0012260000D49401842F6ED
:10235000E061401A290407D041783170017871702A
:10236000801C6D1EB61CF5E71046FEBD08490870BE
:102370002046FEBD6F170000581B000028020020F9
:10238000F80B0020AC060020081800000718000019
:1023900033020020320200208C02002001000020C5
:1023A000000000206C0200203902002010B5034616
:1023B000481E81B20120084CA1420BD38918074C5A
:1023C000A14207D80020110404D058701870521E82
:1023D0009B1CF8E710BDC046B80B0000BC0B00000A
:1023E000FCB50191016A0090446A00252E46202D1B
:1023F0000CD01746F740FF0705D0019FAF400F23D1
:10240000AB40994339432D1D761CF0E70825002683
:10241000202E0CD01346EB40DB0705D0019BB340C8
:102420000F27B740BC431C43361D6D1CF0E70098D6
:1024300001624462FCBD8162704781617047C16284
:10244000704700690840411E88417047FEB50293FD
:10245000019202680090C56800263746202E10D0F1
:10246000029BFB40DB0709D0019BB3400324B4402F
:10247000A5431D430B46B340A2431A43B61C7F1C21
:10248000ECE700980260C560FEBDF8B5012902D1F5
:102490004168194301E041689943416000908168B7
:1024A000002403202646202C0CD01F46F740FF07AF
:1024B00005D01746A7400546A540A9433943A41CAB
:1024C000761CF0E700988160F8BD000096B00EA879
:1024D00020210D91FDF7E3FEE64C0020E081E08035
:1024E000E549FF270F70099020700620C6433C2065
:1024F0000C9027200B903046099A30B121180C9B84
:10250000CA540B9BCA54401CF7E7FEF71DFFFFF7A8
:1025100095F8FEF7E5F9FEF79FFAFEF7C1F9FEF729
:10252000A1F9FEF7DFF9FEF7A9FBFEF7E5FBFEF7E1
:10253000B5FA41F2C020FEF73FFBFEF757F9FEF770
:10254000DBFCFEF733FC099D6561FEF793FD014658
:102550000095E120430228462A46FFF76BFCFFF76F
:10256000A1FAC54B58780C99605440F2C811C34D7C
:10257000695822463C32D17340F2007141182182E1
:1025800029600821081AC7401F7040F2D810281887
:1025900056B1B849891902684423CA54026C4B23C6
:1025A000CA54001D761CF3E7B5484021FFF743FFEE
:1025B000FEF704FC4B22AF4CA05CAF4D29780840DD
:1025C0000292A054099A22726072A8780840A870FA
:1025D000C0B2FDF7F4FFA878207340F24810A74975
:1025E00008180590A748C01C0490A74844F20001B1
:1025F000FFF727FF002800D19CE0FFF779FC9D49F9
:10260000087930B109980871012048210822FEF7A5
:1026100055FD9E480078002854D009999B480170C8
:102620000498082913D08A000EAB9A1800231824A6
:102630001D46042B07D0F8262640C75CB7407D19FD
:10264000F8345B1CF5E71560001D491CE9E70A201A
:102650000E99B1FBF0F1894B99601A46C8322833C4
:10266000F54CA4780025072D12D019600126AE4044
:102670001768B94202D9F6B2344303E0264203D0C8
:10268000B443E4B2EC4EB4701033121D6D1CEAE793
:102690001199B1FBF0F1E94A51610F99B1FBF0F3E7
:1026A000E4498C691A1B0021A34200D20A46E34B7D
:1026B000DA60109AB2FBF0F0DE4AD269801A00D2DA
:1026C00008461861FEF706F828B1FEF70BFCFDF787
:1026D000D1FE00F01DFBDB490878D84EB0B30024D2
:1026E0000C702C36D84D059FD24BD348407884428D
:1026F0001AD22888FDF748FFCE4B3060197869B1AF
:102700000122A240997A3B68984202D91143C94BF1
:1027100003E00A42C74B01D091439972002001C5E2
:1027200010363F1D641CE0E7C3488078997A014366
:10273000D9720DE02346607A217A0A90089181428D
:1027400056D11878002800D0B0E0ADE0B94BD97A66
:1027500008060ED01A7BC8B2904214D05A7A8A4327
:102760005A72FDF72CFFB34B18460C3019460B314B
:1027700007E0D878597A014305D11846093019463F
:102780004B3109780170D8794101B04A5258002A7A
:1027900000D1F3E0AD4A51184A68412A12D88B683B
:1027A0009200A64CA350AA4C121914469C3C2370CC
:1027B00014469D3C1D0A257014469E3C1D0C257038
:1027C0009F3AD4E0512A00D9A8E08B6892009B4C34
:1027D000A3509F4C12191446AC3C23701446AD3CD8
:1027E0001D0A25701446AE3C1D0C2570AF3ABEE0A4
:1027F0000C981E5CD8780690987803900024904935
:10280000A64245D01D190D982A5C6ABB3522AA5CE8
:1028100052BB2F4620372846353007900A98E040B3
:1028200001221040089BE340134083420BD92E2025
:102830002A540698A8B13A704420285C40F2E83245
:10284000504308600FE07B4B0ED20B982A5403983C
:1028500068B13A703D20285C40F2E832504308608D
:1028600002E007980270734B091D641CC8E70798C3
:102870000270F9E730020020000000208C020020E6
:10288000001400487F010020000800487E0100205D
:10289000069808B10020D870039808B100209870FD
:1028A00002980A9919541972012018700C98185C32
:1028B0000024844200D3A0E61D193521695C59B378
:1028C0002846353000260D996E5406700127A74022
:1028D0000B98285C60B12735E0B20121FEF71AFCA5
:1028E0002E70564A40F2C813D158F8B208430DE092
:1028F0002E20285C58B12E35E0B23146FEF70AFC96
:102900002E704E4A40F2C813D05CB843D050FEF748
:10291000A9FE484B0C98185C641CCAE7612A12D8BF
:102920008B689200454CA350494C12191446BC3C8C
:1029300023701446BD3C1D0A25701446BE3C1D0C78
:102940002570BF3A13E0712A32D88B6892003B4C55
:10295000A3503F4C12191446CC3C23701446CD3C76
:102960001D0A25701446CE3C1D0C2570CF3A1B0E57
:102970001370304B01225A7100220A60401CC1B210
:102980001F2900D90020D8711C46FDF79FFE0028A2
:1029900000D12AE6FDF76AFD6079002800D124E61F
:1029A000002060712A4940F20012FDF711FD1CE67B
:1029B000972A0ED0742A11D0962A16D0722A1AD1CC
:1029C0000A7A1D4B1B781340214A5370194A5372DF
:1029D000CFE700225A721E4C6270CBE70A7A164B80
:1029E0001B7813401A4AD370C3E7134A1278184C65
:1029F00062705A72BEE7852A0CD88B68DCB29500EB
:102A00000E4E7451124C1419713C2370094C12195A
:102A1000393AADE7952AADD88B68DCB29500074E00
:102A200074510B4C1419713C2370024C1219423A28
:102A30009EE7C04630020020000000208C020020EB
:102A400018010020480100205C010020AC06002095
:102A5000AC050020B0B542B2002A05D403231446C9
:102A60009C43104BE31803E00C2313400C4C1B1940
:102A70009407E40E8907090EA140FF25A5401C68B4
:102A8000AC430C431C60002A09D41F2101400122E1
:102A90008A40C00804494018032188430260B0BD41
:102AA00014ED00E000E400E000E100E0024A0A402A
:102AB000024302480260704780FFFF1F08ED00E0FC
:102AC00040B1072803D0012803D102207047062017
:102AD00070470420704700220B0404D003789A1832
:102AE000401C491EF8E75042C0B270476E490A6860
:102AF0004CF200039A430A60CA6A2C4B1340CB6223
:102B0000092851D8820001A39A18974600F012B8FC
:102B100000F015B800F01DB800F01EB800F01FB8A6
:102B200000F021B800F023B800F025B800F032B86A
:102B300000F025B801200004CA6A824303E00120A6
:102B40000004CA6A0243CA62C86A40F20012904393
:102B500029E00868086022E00868086014E0086856
:102B600044F2000219E0086844F200020AE0086832
:102B700048F2000211E0086848F2000202E008682A
:102B80004CF2000202430A600120C007CA6A0243F5
:102B9000CA6204E008684CF2000202430A60CA6A92
:102BA00040F200101043C8627047C046FFFEFE7F2F
:102BB000F8B53D4A11680C240C403C4B082C1C46CF
:102BC00018D111688902090F0F2901D08C1C00E06F
:102BD000102415682D0101D511310C461168C90367
:102BE00001D4334905E0916A0F250D40691CB3FB00
:102BF000F1F14C43156813681168052841D800931A
:102C00002D062D0F2BA77F5D2546FD408904490F1A
:102C10002C4F7B5C2946D940830001A6F3189F46C0
:102C200000F00AB800F00FB800F008B800F039B8AA
:102C300000F00BB800F011B8214632E000984005D2
:102C4000400F385CC54029462BE0D06AC0051AD435
:102C5000D06AC00320D51D4923E0D06A800720D068
:102C6000D16A03200140012921461AD0D36A0340CA
:102C700048F20001022B14D0D16A014003290B490C
:102C80000FD000210DE010680004800FD26A002AE6
:102C900004D4B1FBF0F104E00B4902E0401CB5FBA9
:102CA000F0F10846F8BDC0460410024000127A0058
:102CB00000093D00000000000000000001020304C4
:102CC0000607080998380008809FD500003FAB012F
:102CD0001F21014001228A4080090C4943581343B7
:102CE000435070471F21014001228A408009074953
:102CF00043589343435070471F21014001228A40AB
:102D00008009024943581343435070470010024062
:102D1000B0B51348417803290BD80246143200237A
:102D2000102B16D0C418648815682C1910C29B1C6F
:102D3000F6E70021417014220A4B342A0CD0845843
:102D4000A4081D88641B00D20C4684509B1C121DD5
:102D5000F3E7491C4170B0BD01210170B0BDC04610
:102D6000480100207C0200204162704710B5154CDC
:102D70004649884213D01449884212D0EE4988420D
:102D800011D03F49884213D03F4988420DD0404975
:102D900088420CD03B49884213D1F63408E0E41D48
:102DA00006E0F93404E0FD3402E0641D00E0A41DF7
:102DB0002046FFF7A1FF204610BC02BC8E46FFF75D
:102DC00091BF10BD0B0300000010004001680122FC
:102DD000914301607047016801220A430260704715
:102DE00010B50A888262264A904202D0254B98424A
:102DF00019D103687024A34303604B8804681C4303
:102E000004608B8804681C4304608B68C362904232
:102E10000BD1136840F20034A3431360CB881468CD
:102E20001C43146024E08B68C362164B98420BD09D
:102E3000CD4B984208D0144B984205D0134B984282
:102E400002D0134B984215D1036840F20034A343DB
:102E50000360CB8804681C430460904208D00A4A8F
:102E6000904205D00A4A904202D0084A904201D1CD
:102E7000097B0163416901220A43426110BDC046DA
:102E8000002C014000040040004001400048014087
:102E900000440140C2688A43C2607047C2680A4366
:102EA000C260704702698A4302617047C2680A4083
:102EB000531E9A4100690840411E884110407047E6
:102EC0000349002202730260426081607047C0467D
:102ED000FFFF0000F0B5FF22094B0A4C15460E0417
:102EE00009D0EDB206786E409F5DA55D5540401C4F
:102EF000491E3A46F3E7E8B21102081880B2F0BD65
:102F00009837000898360008B0B50D4604467E484C
:102F1000844204D02048844205D1022000E00520EC
:102F2000FFF746FE00E000202168090405D4690887
:102F30004018B0FBF5F080B209E069084000401885
:102F4000B0FBF5F0034901400007400F4018E06076
:102F5000B0BDC046F0FF0000416A0348084070471A
:102F6000014A0A4082627047FF01000010B56649BD
:102F7000884204D0084988420BD1084C00E0054C37
:102F80002046FFF7B9FE204610BC02BC8E46FFF774
:102F9000A9BE10BD0E030000004400401104000053
:102FA000016801220A43026070471F220A40012182
:102FB0009140026A0A43026270471F220A4089094F
:102FC0000958D1400120084070471F220A400123C0
:102FD000934089090A589A430A5070471F220A40B1
:102FE0000123934089090A581A430A507047000088
:102FF000084A914206D1D021425848F200039A4330
:1030000042507047C902C90E01228A40016A114329
:103010000162704709340F341F220A400B049B0DD4
:103020001B58D3408A0D1258C802C00EC2401A4025
:10303000012010407047026801239A430260026831
:1030400040F200639A43026002680A4302607047DC
:10305000026804239A43026002680A4302607047D0
:10306000026801239A430260426843F200039A43D4
:10307000426042680A4342607047026808239A43EC
:10308000026002680A4302607047026801239A43A3
:103090000260026841F200039A43026002680A4338
:1030A0000260704770B50E460921CC06D04D05214F
:1030B000012808D12846FFF791FF204640F2001171
:1030C000FFF7B9F907E02846FFF77FFF204640F2F7
:1030D0000011FFF7B2F906212846012E09D1FFF7AA
:1030E0007DFF204640F2001170BC04BC9646FFF7FD
:1030F000A4B9FFF76AFF204640F2001170BC04BC7F
:103100009646FFF798B9C04600380140B0B5164C56
:1031100000212046FFF728FE012520462946FFF71B
:10312000C1FE20462946FFF7B5FE2046B0BC02BCD2
:103130008E46FFF74BBEC04600200040B0B50A4C9B
:1031400000212046FFF710FE012520462946FFF703
:10315000A9FE20462946FFF7A1FE2046B0BC02BCCE
:103160008E46FFF738BEC04600200040BCB53A4D41
:10317000A87800286AD101A800F032F96878002404
:1031800078B1022818D001285ED1FFF7D7FF01A837
:1031900000780D2828D000243A2828D1EC70AC8083
:1031A00052E001A800783A284ED1FFF7C7FF00246B
:1031B000AC80EC70012018E001A8007829788842E2
:1031C00008D1FFF7A3FF00206870012000F000F98C
:1031D000044639E000243A2810D1EC70AC8001207C
:1031E0006870FFF7ABFF2FE0022068702CE001460B
:1031F0004139C9B2062903D3E14303E06C7023E0EF
:10320000014637393038C2B20A2A00D30846E97875
:1032100001290AD0C1B9A988FF2911D8A9880001BC
:10322000EA4A50540120E8700EE0A988E74A535C4E
:1032300003435354A888401CA8800024EC7003E08A
:1032400000246C70FFF762FF2046BCBD03A0564906
:10325000E322FEF71BFAC046C001002065536E64EE
:103260005374617465203D3D2053544154455F546F
:10327000585F49444C45000080B543484178491E99
:10328000012902D80021417005E04178012902D0CE
:103290004078022803D1FFF739FF002080BD0348A2
:1032A000414940F2A712FEF7F1F9C046A0380008E4
:1032B00070B5354E707800285FD1B07804283ED8BC
:1032C000810001A251188F4600F008B800F025B81F
:1032D00000F009B800F029B800F012B80120002170
:1032E000FFF7E0FE2BE0F08820B3F078012828D02B
:1032F00028BBB0680078410905292AD3372129E085
:103300000024B470032000F063F805460120214634
:10331000FFF7C8FEB470284670BD3A2000F0DAF816
:103320000220B0700020F07009E0307800F0D2F890
:10333000042003E00D2000F0CDF80320B070002041
:1033400070BDB06801780F2008400A2808D33721E3
:1033500007E030210009081800F0BCF80120E2E77E
:103360003021081800F0B6F80020F070B068401C5A
:10337000B060F088401EF080E1E704A00A4940F206
:103380004F12FEF783F9C046C001002065526376F4
:103390005374617465203D3D2053544154455F5240
:1033A000585F49444C450000E43800080B490A784E
:1033B000012A05D14A780270002008700120704768
:1033C0000020704705480021017001207047C04669
:1033D00002494870012008707047C046CC010020A7
:1033E00010B504463F48FFF7B7FD2070012010BD1F
:1033F00000380140FEB502911B2000252946FFF749
:1034000029FB3148FFF764FC0920C6060124304639
:10341000214640F20022FEF7E3FF022101913046EF
:10342000224640F20023294FB847294F304629460B
:10343000224640F20023B8473046214640F200427F
:10344000FEF7CEFF30460199224640F200431F4F5F
:10345000B84730462946224640F200431C4FB84741
:10346000304621462A4640F20013184FB84703223F
:103470003046294640F20013154EB0471248FD3041
:10348000FFF726FC174E3046FFF770FD30460299D5
:10349000FFF73AFD30462946FFF7E2FD3046294660
:1034A000FFF7F3FD30462946FFF7C5FD04213046FE
:1034B000FFF7CEFD08213046FFF7DFFD3046FFF76E
:1034C0006FFD2046FEBDC046110500004D240008DA
:1034D0008B24000880B501460248FFF741FD01201A
:1034E00080BDC046003801407FB5054640F20870F7
:1034F000FFF7EEFB104C2046FFF738FC6E463046D7
:10350000FFF7DEFC0D483080681E0290002001901D
:1035100020463146FFF764FC012520462946FFF787
:10352000BDFC13202946FFF795FA2046FFF753FC10
:10353000284604B070BDC046002000400F0E0000B9
:103540001CB51A4C607858BB01A8FFF749FF2078DA
:10355000032823D8810001A251188F4600F01CB81F
:1035600000F004B800F00CB800F016B8002060803D
:103570006088411C61801549019A0A5402200AE0C2
:103580006088FF2806D86088411C61800F49019A35
:103590000A5401E003202070FFF7D0FD00201CBD7D
:1035A00003A03C49F022FEF771F8C046F401002068
:1035B00065536E645374617465203D3D20535441DE
:1035C00054455F54585F49444C450000F40A0020BC
:1035D000B0B5284D287828B10024032805D002284A
:1035E00009D10120FFF7F4FE0446FFF78FFD01200B
:1035F00028702046B0BD28780028F6D02878022808
:10360000F3D028780328F0D00248224940F265120E
:10361000FEF73CF80239000870B5164E30780128E4
:1036200022D17078012805D080B901200021FFF750
:1036300039FD0BE0B08858B1B0680078FFF74AFF59
:10364000B068401CB060B088401EB080002070BDE3
:103650000320FFF7BDFE0446012000252946FFF7A1
:1036600021FD7570204670BD03A00A4940F22B125F
:10367000FEF70CF8F4010020655263765374617410
:1036800065203D3D2053544154455F52585F4944A5
:103690004C4500006539000800C1814001C08041EF
:1036A00001C0804100C1814001C0804100C1814012
:1036B00000C1814001C0804101C0804100C1814002
:1036C00000C1814001C0804100C1814001C08041F2
:1036D00001C0804100C1814001C0804100C18140E2
:1036E00000C1814001C0804100C1814001C08041D2
:1036F00001C0804100C1814000C1814001C08041C2
:1037000001C0804100C1814001C0804100C18140B1
:1037100000C1814001C0804101C0804100C18140A1
:1037200000C1814001C0804100C1814001C0804191
:1037300001C0804100C1814000C1814001C0804181
:1037400001C0804100C1814001C0804100C1814071
:1037500000C1814001C0804100C1814001C0804161
:1037600001C0804100C1814001C0804100C1814051
:1037700000C1814001C0804101C0804100C1814041
:1037800000C1814001C0804100C1814001C0804131
:1037900001C0804100C1814000C0C101C30302C219
:1037A000C60607C705C5C404CC0C0DCD0FCFCE0E81
:1037B0000ACACB0BC90908C8D81819D91BDBDA1AF1
:1037C0001EDEDF1FDD1D1CDC14D4D515D71716D661
:1037D000D21213D311D1D010F03031F133F3F232D1
:1037E00036F6F737F53534F43CFCFD3DFF3F3EFE41
:1037F000FA3A3BFB39F9F83828E8E929EB2B2AEAB1
:10380000EE2E2FEF2DEDEC2CE42425E527E7E62620
:1038100022E2E323E12120E0A06061A163A3A26290
:1038200066A6A767A56564A46CACAD6DAF6F6EAE00
:10383000AA6A6BAB69A9A86878B8B979BB7B7ABA70
:10384000BE7E7FBF7DBDBC7CB47475B577B7B676E0
:1038500072B2B373B17170B0509091519353529250
:1038600096565797559594549C5C5D9D5F9F9E5EC0
:103870005A9A9B5B99595898884849894B8B8A4A30
:103880004E8E8F4F8D4D4C8C4484854587474686A0
:103890008242438341818040000000000102030412
:1038A0002820655263765374617465203D3D205332
:1038B000544154455F52585F5243562029207C7C26
:1038C000202820655263765374617465203D3D2045
:1038D00053544154455F52585F574149545F454FD7
:1038E000462029002E2E2F4170702F4D6F64627577
:1038F000732F61736369692F6D6261736369692EE8
:1039000063002820655263765374617465203D3DE1
:103910002053544154455F52585F494E4954202921
:10392000207C7C2028206552637653746174652066
:103930003D3D2053544154455F52585F52435620F9
:1039400029207C7C2028206552637653746174653D
:10395000203D3D2053544154455F52585F455252DB
:103960004F522029002E2E2F4170702F4D6F646210
:1039700075732F7274752F6D627274752E630000EB
:10398000A03900080000002090000000100100088D
:10399000303A000890000020381B00002C0100087D
:1039A000FF07FF0000A24A0402000000110000000F
:1039B000F11C000804000000F71B000803000000D1
:1039C000A11B000810000000E11D00080600000017
:1039D000551D000817000000551C000801000000DC
:1039E000C91A000805000000111D00080F000000A2
:1039F000871D000802000000351B000800000000C1
:103A000000000000000000000000000000000000B6
:103A100000000000000000000000000000000000A6
:103A20000000000000000000000000000000000096
:04000005080000CD22
:00000001FF
